:100000000C941A020C946D020C946D020C946D0207
:100010000C946D020C946D020C946D020C946D02A4
:100020000C946D020C946D020C94DE2A0C946D02FB
:100030000C94B52A0C946D020C946D020C946D0214
:100040000C946D020C946D020C946D020C946D0274
:100050000C946D020C945B2E0C946D020C946D024A
:100060000C946D020C946D020C946D020C946D0254
:100070000C946D020C946D020C946D020C946D0244
:100080000C946D020C946D020C946D020C946D0234
:100090000C946D020C946D020C946D020C946D0224
:1000A0000C946D020C946D020C946D020631FF09E4
:1000B00074A1010975150026FF00952075088102BD
:1000C0000976150026FF00952075089102C00501EC
:1000D0000902A1010901A1008501050919012908E9
:1000E00015002501950875018102050109300931C6
:1000F0001581257F95027508810609381581257FB0
:10010000950175088106050C0A38021581257F9531
:100110000175088106C0C005010980A1018502168C
:1001200001002637001A81002AB700751095018159
:1001300000C0050C0901A1018503160100269C02DF
:100140001A01002A9C02751095018100C005010961
:1001500006A101050719E029E71500250195087595
:10016000018102950175088101050819012905958C
:100170000575019102950175039101050719002983
:10018000FF150026FF00950675088100C073706595
:1001900065643A2025730A007573625F7374617435
:1001A000653A20253032580A00686F73742E546106
:1001B000736B3A2025640A00526F6C6C6F7665721F
:1001C000206572726F723A2069676E6F7265640D96
:1001D0000A002069676E6F7265640D0A000D0A00DF
:1001E000202530325800696E7075742025643A00FD
:1001F0000A4C6F6F702073746172742E0A000A5576
:10020000534220636F6E666967757265642E0A00DB
:100210000A544D4B3A3632653939352F4C554641E3
:100220003A6436613764662F554853323A3835613F
:100230006637360A0009025400030100A03209049F
:100240000000010301010009211101000122400009
:100250000705810308000A090401000103010200E7
:10026000092111010001227F000705820308000116
:10027000090402000103000000092111010001220C
:100280002200070583032000011201100100000075
:1002900008EDFE5B001508010200013C0355005308
:1002A000004200200074006F0020005500530042FF
:1002B0000020006B006500790062006F0061007231
:1002C000006400200063006F006E0076006500721D
:1002D000007400650072000000080354004D004BDC
:1002E00000000004030904808080800405060708DC
:1002F000090A0B0C0D0E0F101112131415161718F6
:10030000191A1B1C1D1E1F202122232425262728E5
:10031000292A2B2C2D2E2F303132333435363738D5
:10032000393A3B3C3D3E3F404142434445464748C5
:10033000494A4B4C4D4E4F505152535455565758B5
:10034000595A5B5C5D5E5F60616263646573676898
:10035000696A6B6C6D6E6F70717273808080808063
:1003600080808080808003020180808066807500AC
:1003700074767780808080767780808080808080AF
:10038000808080808080808080808080808080806D
:10039000808080808080808080808080808080805D
:1003A000808080808080808080808080808080804D
:1003B000808080808080808080808080808080803D
:1003C0008080808080808078797A7B7C7D7E7F8051
:1003D000808080808080808080808080808080801D
:1003E00080808080808080290A002575002F00256C
:1003F00075005D280025640020002564002000258C
:10040000640020002564007C0025303258006D6FA8
:100410007573656B6579205B62746E7C78207920DA
:100420007620685D287265702F61636C293A205BC5
:100430000000C32911241FBECFEFDAE0DEBFCDBF1D
:1004400004B603FE28C08091E5059091E605A091D1
:10045000E705B091E8058730904BA740B04BD9F441
:100460001092E5051092E6051092E7051092E80556
:1004700014BE0FB6F894A8958091600088618093AF
:100480006000109260000FBE1092010810920008E8
:10049000E0E0F8E3099511E0A0E0B1E0E0E2F0E689
:1004A00002C005900D92AA39B107D9F725E0AAE953
:1004B000B1E001C01D92A53EB207E1F712E0CAE12A
:1004C000D2E004C02197FE010E94F42FC931D10768
:1004D000C9F70E94DA2B0C940E300C940000FF93A5
:1004E000EF93E0919A01F0919B01309709F0099503
:1004F000EF91FF910895FC018591803011F0EFDFBD
:10050000FBCF0895FF27E0E230E247FF0CC04195A2
:1005100097FF09C0EDE26095709580959095611DFB
:10052000711D811D911D27FF02C0219530E350E20E
:10053000AA27660F771F881F991FAA1FA41710F0FC
:10054000A41B63955A95A9F7AA3008F0A95FA05D8E
:10055000AF93F395611571058105910541F7ED3272
:1005600011F4EF93F395F21718F43F93F395FBCF43
:100570008F91B5DFFA95E1F70895E991F9918591A9
:10058000803021F0853219F0AADFF9CF089520E0FC
:10059000E89455915532C1F3503311F46894559154
:1005A0005A3348F4505390F3220F022E220F220F99
:1005B000200D250FF4CF0EF4219589919991533692
:1005C00019F3533729F1533559F1BC01882799277D
:1005D000E8945C3621F48991999168945591543648
:1005E00039F446EF7EF077FF0DC08FEF9FEF0AC022
:1005F00055374AE039F0583540E121F0523642E0B3
:1006000009F00895FF93EF937DDFEF91FF91B7CF4E
:10061000FF93EF93FC0181918030B9F360DFFBCF52
:10062000FF93EF9368DFF1CFDF93CF93CDB7DEB7C2
:100630002596A3DFCF91DF910895FC018EE695E02A
:100640009583848381E491E0918380838FE591E0B9
:1006500093838283108E118E128E138E148E168EBB
:1006600081E0878B168A148A178288E080878CE362
:1006700081871286138684E084871586168687878D
:10068000108A118AA4ECB5E090E080E02D913D91B4
:10069000232B41F4880F991FDC01AC53BA4FED9323
:1006A000FC93089501968031910581F70895803F6C
:1006B000C1F480914B0487FD10924B0480914A0451
:1006C00081110EC080914B0481110AC080914C04AD
:1006D000811106C080914D04811102C01092430423
:1006E0000895813F29F480914B0418162CF3E6CF2E
:1006F00090914A04823F29F497FFE0CF10924A0478
:10070000DDCF833F19F41916CCF3D8CF893F39F4E4
:1007100080914C04181694F610924C04CFCF8A3F67
:1007200029F480914C0487FFC9CFF6CF8B3F39F471
:1007300080914D0487FFC2CF10924D04BFCF8C3FF4
:1007400029F480914D041816BCF3B8CF843F31F4DE
:10075000809149048E7F80934904B0CF853F21F476
:10076000809149048D7FF7CF863F21F48091490421
:100770008B7FF1CF873F21F480914904877FEBCFB6
:10078000883F21F4809149048F7EE5CF8D3F31F47D
:10079000809142048E7F8093420490CF8E3F21F45B
:1007A000809142048D7FF7CF8F3F09F087CF8091F2
:1007B00042048B7FF0CF8091420480FD16C081FD02
:1007C00016C082FD16C0809143048823A1F08832B0
:1007D00080F428E0829FC001112468E270E00E944A
:1007E000E02F862F672B39F0089582E0089584E08A
:1007F000089588E0089581E008958091420480FD85
:1008000014C081FD14C082FD16C08091430488236A
:1008100081F0843180F422E3829FC001112464E1DD
:1008200070E00E94E02F862F08958CE0089589E102
:10083000089585E0089582E30895803F31F40E9491
:10084000FD03819580934B040895813F19F40E9424
:10085000FD03F8CF823F31F40E94FD038195809320
:100860004A040895833F19F40E94FD03F8CF893F9D
:1008700029F40E94DB0380934C0408958A3F21F4FD
:100880000E94DB038195F7CF8B3F31F40E94DB039D
:10089000819580934D0408958C3F19F40E94DB03E9
:1008A000F8CF843F31F480914904816080934904FA
:1008B0000895853F21F4809149048260F7CF863FF7
:1008C00021F4809149048460F1CF873F21F4809125
:1008D00049048860EBCF883F21F48091490480610E
:1008E000E5CF8D3F31F480914204816080934204D2
:1008F00008958E3F21F4809142048260F7CF8F3FAC
:10090000B9F7809142048460F1CF20E1729FF00139
:100910001124E60FF11DE951FD4F6491E62FE29598
:10092000E77028E0829FC00111248E0F911D24E002
:10093000880F991F2A95E1F7E62FEF70E80FF92F3E
:10094000F11DEE0FFF1FE050F84985919491089535
:10095000ECE9F2E09281891301C01282319692E0B3
:10096000E23AF907B9F70895AEE9B2E0EFEF90E0A7
:100970002D91821751F0EF3F19F4211101C0E92F99
:100980009F5F9630A9F7EF3F09F408950E2E000CF3
:10099000FF0BE456FD4F8283089580913C049091B3
:1009A0003B04892B80939C0290913A04992381F017
:1009B000892B80939C02EDE9F2E080E09191911106
:1009C0008F5F92E0E43AF907C9F7811110923A0477
:1009D000E0914504F0914604309731F00280F381B4
:1009E000E02D8CE992E0099408954F925F926F9206
:1009F0007F929F92AF92BF92CF92DF92EF92FF923F
:100A00000F931F93CF93DF9300D000D01F92CDB7E9
:100A1000DEB76B837C838D837A018C819D81892BEA
:100A200049F08FEFF81204C081E09FEF491719F0E9
:100A300080E001C081E080FD6AC00F2D10E0CE2C67
:100A4000D12C8B81882309F456C0409036035090F6
:100A5000370360903803709039038091320390918E
:100A60003303A0913403B0913503482A592A6A2AE6
:100A70007B2A2FE1A22EB12C9A2CD301C2010A2C81
:100A800004C0B695A795979587950A94D2F780FDEF
:100A90002BC081E0A81AB10878F7912CF80194E0F6
:100AA000EE0FFF1F9A95E1F7E65CFC4FEC0DFD1D84
:100AB0009082E982FA8269817A81892D0F900F9064
:100AC0000F900F900F90DF91CF911F910F91FF909A
:100AD000EF90DF90CF90BF90AF909F907F906F90FE
:100AE0005F904F900C948504B7018A2D0E94850475
:100AF000019779F2D3CFF80184E0EE0FFF1F8A95BA
:100B0000E1F7E65CFC4FEC0DFD1D9080D2CF90E04C
:100B100080E00F900F900F900F900F90DF91CF918A
:100B20001F910F91FF90EF90DF90CF90BF90AF900B
:100B30009F907F906F905F904F90089541E050E0BC
:100B400060E070E004C0440F551F661F771F8A9550
:100B5000D2F74095509560957095809136039091AD
:100B60003703A0913803B091390384239523A6233A
:100B7000B7238093360390933703A0933803B09341
:100B80003903089541E050E060E070E004C0440F94
:100B9000551F661F771F8A95D2F780913603909173
:100BA0003703A0913803B0913903842B952BA62BE2
:100BB000B72B8093360390933703A0933803B093F9
:100BC000390308958091310390910003981301C077
:100BD00008958F5F8770FACF1F93CF93DF9300D074
:100BE00000D01F92CDB7DEB7942F4983252F5A83AB
:100BF0006B837C838D834C815D8181E0452B31F05B
:100C00002F3F19F481E09F3F09F080E0182F117009
:100C100080FD2CC049815A816B817C818D810E942D
:100C2000F504292F22952F702C3078F42A30A8F45F
:100C300022502230C8F0812F0F900F900F900F900C
:100C40000F90DF91CF911F9108952C3011F02F302C
:100C500091F793FB112710F9EECF803C28F0803EEE
:100C600050F3815F833038F311E0E5CF10E0E3CF3C
:100C7000882341F0809590913C04892380933C0423
:100C80000C94CD040895882339F090913C04892B6D
:100C900080933C040C94CD0408952091F802309187
:100CA000F9022817390771F09093F9028093F8023E
:100CB000E0914504F0914604309721F00084F185DD
:100CC000E02D099408952091F6023091F70228173B
:100CD000390771F09093F7028093F602E091450492
:100CE000F0914604309721F00680F781E02D0994B9
:100CF0000895E0914504F0914604309721F0019069
:100D0000F081E02D099480E00895E8EDF0E0808125
:100D10008E7F80831092E2001092DA001092E10040
:100D2000A0EEB0E08C9181608C9380818F7780837E
:100D300019BCA7EDB0E08C918E7F8C9380818F7E63
:100D400080831092DE0208950E948506F89487E75A
:100D500097E7909301088093000887E090EBDC010F
:100D60008093E5059093E605A093E705B093E80529
:100D700088E19CE00FB6F894A895809360000FBEC0
:100D800090936000FFCFFC018091F3029091F402F8
:100D900086179707A0F06115710529F49091E80076
:100DA0009E779093E80090E06115710551F49111E0
:100DB00008C08091E80082FF35C080E00895BC0142
:100DC000F2CF8091F5028823C9F18530C9F1809175
:100DD000E80083FD31C08091E80082FDEACF809178
:100DE000E80080FFE1CF2091F3008091F200322FE4
:100DF000282F6115710519F02830310558F091E060
:100E00002830310509F090E02091E8002E772093FA
:100E1000E800CACF81918093F100615071092F5F82
:100E20003F4FE7CF8091F502882341F0853041F0B4
:100E30008091E80083FFBDCF81E0089582E00895AE
:100E400083E008952091E4003091E50085E69091DB
:100E5000EC0090FF06C09091E80090FF06C080E093
:100E600008959091E80092FDFACF9091F5029923B0
:100E700091F0953091F09091EB0095FD10C040916C
:100E8000E4005091E5002417350709F381509A01D9
:100E9000F1F684E0089582E0089583E0089581E00A
:100EA00008958091ED0287FF13C08091E80082FFD2
:100EB00006C08091E8008B778093E80004C08091A1
:100EC000F5028111F2CF08958091F5028823D9F3BC
:100ED0008091E80080FFF8CF8091E8008E77ECCF1A
:100EE000982F9093E900242F762F50E0891731F046
:100EF0007091EC002091ED005091F00021FD07C0B1
:100F00009F5F973071F78093E90081E008953091F9
:100F1000EB003E7F3093EB003091ED003D7F30934E
:100F2000ED003091EB0031603093EB007093EC00FA
:100F30002093ED005093F0002091EE0027FDE0CFCC
:100F400080E008950F931F93CF93DF93CDB7DEB763
:100F5000AA970FB6F894DEBF0FBECDBF8091F50201
:100F6000882309F44EC11091E9001F708091EC00B4
:100F700080FF39C080E8182B1092E9008091E800CA
:100F800083FF3CC1EDEEF2E085EF92E02091F100AD
:100F900021938E179F07D1F78091EE02833009F4D9
:100FA00070C018F5813009F447C0823009F4DAC006
:100FB0008091E80083FF14C18091ED029091EE02D0
:100FC0009A3008F00DC1E92FF0E0E751F84F0C948A
:100FD000F42FC308E908F008E908F0084B096D0987
:100FE000F0086C0A790A80E0C6CF8A3009F4A9C0FB
:100FF0008B3009F47DC08930D9F68091ED028132C1
:10100000B9F68091F1029091F202892B89F68091D4
:10101000E800877F8093E8008091E80082FF2CC081
:101020008091F1008093E1028091E8008B778093BA
:10103000E8000E945107BCCF8091ED02813A09F08F
:10104000B7CF8091E800877F8093E8008091F1021C
:101050009091F202892B61F060E090E080E070E016
:101060000E94C3068091E8008B778093E800A0CFB0
:1010700068E082EE92E0F3CF8091F5028111CCCF4F
:1010800097CF8091ED02813A09F092CF8091F102E1
:101090009091F202892BA1F48091E800877F8093E0
:1010A000E8008091E80080FFFCCF809111018093DF
:1010B000F1008091E8008E778093E8000E9451074C
:1010C0008091F1029091F202019709F071CF809125
:1010D000E800877F8093E8008091E80080FFFCCFE4
:1010E000809110018093F1008091E8008E779FCF6E
:1010F0008091ED02813209F05BCF8091F1029091F5
:10110000F202892B59F48091E800877F8093E800F0
:101110000E9451078091EF02809311018091F102AA
:101120009091F202019709F043CF8091E800877F08
:101130008093E8000E9451078091EF028093100194
:1011400037CF8091ED02813209F032CF8091E800F3
:10115000877F8093E8000E9451078091F00280937E
:10116000E00226CF8091ED02813A09F021CF8091F3
:10117000E800877F8093E8008091E80080FFFCCF43
:101180008091E002AFCF803889F0823849F58091B4
:10119000F1028F70873020F58093E9008091EB0099
:1011A00085FB882780F91092E90006C08091EA0249
:1011B0009091EB02911182609091E800977F90935B
:1011C000E8008093F1001092F1008091E8008E77A2
:1011D00031C0282F2D7F21F48823F1F0823079F15E
:1011E0008091E80083FF0AC08091E800877F8093A8
:1011F000E8008091EB0080628093EB001F701093F9
:10120000E900AA960FB6F894DEBF0FBECDBFDF91FE
:10121000CF911F910F9108958091EF02813001F7D6
:10122000933009F080E08093EB021092E900809106
:10123000E800877F8093E8000E945107D1CF80911A
:10124000EF028111F2CF8091F1028F702FEF280F02
:10125000263030F68093E9002091EB0020FFE5CFA7
:10126000933031F48091EB0080628093EB00DDCF0E
:101270009091EB0090619093EB0021E030E001C091
:10128000220F8A95EAF72093EA001092EA008091F3
:10129000EB008860EACF8111A3CF0091EF020F77B6
:1012A0008091E3008078802B8093E3008091E800B8
:1012B000877F8093E8000E9451078091E80080FFBB
:1012C000FCCF8091E30080688093E30083E001110C
:1012D00001C082E08093F50283CF8058823008F00D
:1012E0007FCF2091EF023091F0022C3D83E0380750
:1012F000A1F583E08A838AE289834FB7F894DE01FF
:10130000139620E03EE051E2E32FF0E050935700C7
:10131000E49120FF03C0E295EF703F5FEF708E2FE6
:1013200090E0EA30C0F0C7968D939D932F5F2431F3
:1013300059F74FBF8091E800877F8093E8006AE209
:1013400070E0CE0101960E94C3068091E8008B7781
:101350008093E80045CFC096E7CF8091F10290914D
:10136000F202432F55274330510509F44FC078F559
:101370004130510509F445C084E590E0E5E3F2E031
:101380004230510509F02CCF2091E800277F2093AF
:10139000E8002091F3023091F4028217930708F4D9
:1013A0009C0140E02115310509F063C0411161C085
:1013B0008091E80082FDC9CF8091F502882329F24F
:1013C000853019F28091E80083FFF2CFBECF413221
:1013D000510509F43FC04232510509F001CF833075
:1013E000910508F0FDCEFC01EE0FFF1FEF5CFE4FF4
:1013F0000190F081E02D825D9E4FDC018C9190E0A8
:101400001DC082E190E0E9E8F2E0BECF3327213051
:101410003105C1F060F02230310509F0E1CEEBE991
:10142000F2E0E4918E2F90E0EBE9F2E007C0E3EE0A
:10143000F2E0E4918E2F90E0E3EEF2E0009709F401
:10144000CFCEA2CFE9EDF2E0E4918E2F90E0E9ED6E
:10145000F2E0F4CF8330910508F0C2CE880F991FD7
:10146000FC01E95CFE4F0190F081E02D89E090E005
:101470008BCF8091F502882309F467CF853009F47A
:1014800064CF8091E80083FD60CF8091E80082FD09
:101490008FCF8091E80080FF85CF8091F3009091FD
:1014A000F2008927982789272115310519F08830FE
:1014B000910550F041E0089709F040E08091E80084
:1014C0008E778093E8006ECF44914093F10031967F
:1014D000215031090196E8CF803809F081CE809102
:1014E000E800877F8093E8008091EC028093F10010
:1014F0006CCE811175CE0091EF02023008F070CEF3
:101500008091E800877F8093E8000093EC020E94BE
:101510005107002399F084E08093F50242E061ECEA
:1015200081E00E94700742E061EC82E00E94700757
:1015300046E261EC83E00E94700752CE8091E300A6
:1015400087FDE9CF81E0E8CFEF92FF920F931F93E1
:10155000CF937C018B010E942207C82F811119C0F3
:101560008091E80085FD0DC08091E8008E77809322
:10157000E8000E94A2070E942207882389F3C82F4F
:1015800008C0F70181917F018093F100015011099A
:1015900039F78C2FCF911F910F91FF90EF90089505
:1015A000CF92DF92EF92FF920F931F93CF93DF932F
:1015B000C8EDD0E088818F7E8883E7EDF0E0808100
:1015C0008160808384E082BF81E08093DE02888135
:1015D0008E7F888302EE10E0F80110821092DA000C
:1015E00081EEC82ED12CF601108288818F778883F6
:1015F00088818068888388818F7D888319BC109258
:10160000F5021092EC021092EB021092EA0290EEB8
:10161000E92EF12CF70180818B7F808388818160A6
:10162000888342E060E080E00E947007F6018081DC
:101630008E7F8083F80180818160808380818860D3
:101640008083F70180818E7F808388818061888399
:10165000DF91CF911F910F91FF90EF90DF90CF908E
:1016600008958091E10208950F931F93CF93DF9324
:10167000FC018B01EA0180819181892B31F19281FA
:10168000992349F128813981232BF9F0D8012D9133
:101690003C91D9014C918381682F691B770B808124
:1016A0009181860F971FDC014C9382818150828348
:1016B00088819981019799838883D8018D919C9124
:1016C000119701968D939C93DACF80E0DF91CF91B3
:1016D0001F910F9108958381828381E0F7CFCF938B
:1016E000DF93EC018A819B81DC01ED91FC91048008
:1016F000F581E02D6A8509958A85813439F4EA817E
:10170000FB81EA58FF4F80818B7F80831A861B867E
:101710001C861D861E861F86188A80E0DF91CF9169
:10172000089581E0693009F080E00895FC01828528
:101730000895DF92EF92FF920F931F93CF93DF9361
:10174000EC0185E0E62EF12CFE01869FE00DF11DF7
:101750001124908596FF24C0192F177001E085E0B1
:10176000D82E8FEF800F8F3008F001E0602F70E0EF
:10177000062FD69EF001D79EF00D1124EC0FFD1F11
:1017800080858695869586958770181701F16F5F1D
:101790007F4F603168F38D81811302C011501D832A
:1017A00085E08E9DF0018F9DF00D1124EC0FFD1F43
:1017B000108681E0818712862296D783C683DF91C7
:1017C000CF911F910F91FF90EF90DF900895CE0180
:1017D0000E94990BC6CFFC0121E0613499F49C0171
:1017E000255B3F4F61E0AC014E5F5F4F158666871A
:1017F00017865487438735962E173F07B9F7FC01A4
:10180000158208953585631729F02F5F35962031AD
:10181000C9F70895622F0C94990BCF93DF93FC01C5
:1018200067FD12C0283080F4442319F08581873089
:1018300059F0EF01A1E0B0E08D85882349F11196C0
:101840002596A031B105C1F780E018C085E08A9FD8
:10185000E0018B9FD00D1124CE0FDF1F442389F0B0
:1018600081E4888785818F5F858325E02A9FC00179
:101870002B9F900D1124E80FF91F8085DF91CF91E8
:10188000089581E08887F1CF2770687B622B0FC0B5
:101890006623E1F26770660F660F660F4423A1F3BB
:1018A000606485818F5F85838770687F682B25E002
:1018B0002A9FC0012B9F900D1124E80FF91F60870C
:1018C000862FDCCFFC0121E0611102C0069608954D
:1018D0003585631739F02F5F35962031C9F790E0D1
:1018E00080E00895069635E0239F800D911D112418
:1018F00008950F931F93CF93DF932115310599F02E
:10190000E901042F162F0E94620CFC0186ED30972E
:1019100029F01283D183C083038380E0DF91CF91CC
:101920001F910F91089588EDF9CF81E008952FB7A9
:10193000F89460913D0470913E0480913F04909131
:1019400040042FBF0895CF93C091BA02C1110BC0BC
:101950000E94970C643C79408105910520F081E05C
:101960008093BA02C1E08C2FCF9108952FB7F894DD
:1019700080913D0490913E04A0913F04B0914004B9
:101980002FBF0895EF92FF920F931F93CF93DF9392
:10199000D82F0FB607FE46C08091F502843079F04B
:1019A0008091030190E001962091050130E08223AF
:1019B0009323209104012817190609F0D0C00E9432
:1019C000A30C81110FC08091030190E0019620913A
:1019D000050130E082239323209104012817190682
:1019E00009F0BDC00E94B60C8C01C091E900CF7017
:1019F0008091EC0080FD38C080E0C82B83E08093AC
:101A0000E90085E0E82E8091EB0085FD08C080911B
:101A1000EB0080FF04C08091EE0087FD45C0CF70D1
:101A2000C093E900E09103018E2F90E00196209190
:101A3000050130E082239323209104012817190621
:101A400009F460C08091010190910201E80FF92F23
:101A5000F11DD083809103018F5F9091050189234F
:101A60008093030181E074C080E8C7CFE091010159
:101A7000F0910201E80FF11D90818F5F2091050127
:101A80008223809304019093F1008091E80085FD0A
:101A90000BC08091E80080FF07C08091E8008E773E
:101AA0008093E800E092000180910401909103018D
:101AB000981751F19091E80095FDD8CF80E02BC0A8
:101AC0001092F10034C08091030190E001962091C2
:101AD000050130E082239323209104012817190681
:101AE00009F09DCFF0900001FF2009F498CF0E94EB
:101AF000B60C8017910709F486CFFA94F092000192
:101B00008C0181CF80E024C08091E80085FFD6CF92
:101B1000D093F10081E02091F3009091F200322FF8
:101B2000292F232B79F09091E80090FF0BC0909122
:101B3000E80095FDC5CF9091E8009E779093E8006E
:101B4000E0920001882309F4BECFCF70C093E90072
:101B5000DF91CF911F910F91FF90EF900895E09149
:101B6000030170CF0E94C20C80E008958F929F9273
:101B7000AF92BF92CF92DF92EF92FF920E94BC2E63
:101B80004B015C0120E030E04AE755E40E944B2F16
:101B90006B017C0120E030E040E85FE30E94812E91
:101BA00087FD30C020E03FEF4FE757E4C701B601A3
:101BB0000E94462F1816F4F420E030E040E251E491
:101BC000C501B4010E944B2F0E948D2E20E931E007
:101BD0006115710549F4FF90EF90DF90CF90BF90B1
:101BE000AF909F908F900895C9010197F1F76150D0
:101BF0007109EECFC701B6010E948D2ECB0101976E
:101C0000F1F7E9CF61E070E0F9CFEF92FF920F9327
:101C10001F93CF93DF938A01EB017B01E40EF51E46
:101C2000CE15DF0521F089910E94C20CF9CFC801C1
:101C3000DF91CF911F910F91FF90EF900895862F24
:101C40000E94C20C81E090E00895089581E090E048
:101C500008958FEF9FEF089590E080E00895089534
:101C6000EF92FF92CF93DF93FC01E70187898230E7
:101C700028F0948996132CC0823051F5648B458BE3
:101C80009B819370933021F59A8197FF21C09E81AB
:101C9000258D291708F4958F282F30E0D901AA0F38
:101CA000BB1FA20FB31FAE0FBF1F9A819F70179665
:101CB0009C9317979C8118969C93189794E019967B
:101CC0009C932E0F3F1FD90151964C938F5F878BAA
:101CD000DF91CF91FF90EF900895EF92FF920F93D5
:101CE00002970E94300E0F91FF90EF90089570E0E0
:101CF000685F7F4F660F771F860F971FFC018081FB
:101D00009181089581E0613009F080E0089581E0DB
:101D1000633009F080E00895FC0186810895CF9337
:101D2000DF93EC018C819D81DC01ED91FC910480BD
:101D3000F581E02D6E8109951C8A1D8A81E08F8BCB
:101D40001E82188E198E1A8E1B8E1C8E80E0DF91DB
:101D5000CF9108952E9808952E9A08950F931F936A
:101D6000CF93DF93D82FC62F8A010E94AA0ED2608C
:101D7000DEBDF8018C2F882339F00DB407FEFDCFAE
:101D800091919EBD8150F7CFC00FD12FD11D0DB4C1
:101D900007FEFDCF0E94AC0ECE01DF91CF911F91C7
:101DA0000F910895CF93DF93C82FD62F0E94AA0ECC
:101DB000C260CEBD0DB407FEFDCFDEBD0DB407FE83
:101DC000FDCFDF91CF910C94AC0ECF93C82F0E9422
:101DD000AA0ECEBD0DB407FEFDCF1EBC0DB407FE8E
:101DE000FDCF0E94AC0E8EB5CF9108958F929F9239
:101DF000AF92BF92CF92DF92EF92FF920F931F9319
:101E0000CF93DF93882E962E5A010E94970C6B0178
:101E10007C0128E8C20E23E1D21EE11CF11CC0E0C7
:101E200010E000E0D0E098280E94970C6C197D0922
:101E30008E099F0997FF1EC0692D80EF0E94D20E68
:101E40000E94970C6C197D098E099F0997FF09C0A4
:101E500088EC0E94E50E87FFF3CF60E888EC0E94D3
:101E6000D20E88EF0E94E50EC82FCF70C43081F0EB
:101E7000CE30B9F08C2FDF91CF911F910F91FF9051
:101E8000EF90DF90CF90BF90AF909F908F9008958C
:101E90000F5F1F4FA114B10439F20A151B0521F67B
:101EA000E9CFDF5FD33009F0BFCFE4CFAF92BF926D
:101EB000CF92DF92EF92FF920F931F93CF93DF9316
:101EC000EC01B62EA42E69010E94620C7C0186ED05
:101ED000E114F10409F447C0D701ED91FC91119789
:101EE00087ED309709F43FC013969C9180E09817D6
:101EF00031F02081A21629F033968F5FF8CFF0E001
:101F0000E0E0D601ED93FC938BED309761F12281F7
:101F100026952695203108F02FE081E090E0A0E0A2
:101F2000B0E004C0880F991FAA1FBB1F2A95D2F7E3
:101F30000197F801918380836B2D80EE0E94D20E71
:101F400088ED0E94E50ED70114969C91682F697F59
:101F5000992329F0CA58DF4F68816260682B88EDA9
:101F60000E94D20E80E0DF91CF911F910F91FF90E0
:101F7000EF90DF90CF90BF90AF9008959F92AF9277
:101F8000BF92CF92DF92EF92FF920F931F93CF9366
:101F9000DF936C01C42FD22F99249394E62EF12C59
:101FA000EE0CFF1CE80EF91E86E5E80EF11CA42ECF
:101FB000B12CABE2AA0EB11CAA0CBB1CAC0CBD1C14
:101FC000F70180819181DC01ED91FC910280F38128
:101FD000E02D202F4D2F6C2F0995182F803E09F0F2
:101FE00066C0C11158C061E088EE0E94D20E88EE32
:101FF0000E94E50E80FDFBCF60E488EC0E94D20ECB
:1020000088ED0E94E50E682F686088ED0E94D20E70
:1020100088EC0E94E50E86FFFBCF66E670E080E06C
:1020200090E00E94B60DF70180819181DC01ED9175
:10203000FC910190F081E02D202F4D2F6C2F099500
:10204000182F8D3009F051C08FEF890D8330A8F122
:10205000C1114EC061E088EE0E94D20E88EE0E944F
:10206000E50E80FDFBCF60E488EC0E94D20E88ED87
:102070000E94E50E682F686088ED0E94D20E88EC01
:102080000E94E50E86FFFBCF66E670E080E090E000
:102090000E94B60D1DC0F50180819181DC01ED919A
:1020A000FC910284F385E02D6D2F0995BCCF8D3016
:1020B00061F48FEF890D833058F464E670E080E0BE
:1020C00090E00E94B60D93947BCF882309F4ABCFA8
:1020D000812FDF91CF911F910F91FF90EF90DF90B3
:1020E000CF90BF90AF909F900895882389F3B0CF91
:1020F0008C2F90E08B96880F991F8C0D9D1DFC01F5
:1021000080819181DC01ED91FC910284F385E02DC9
:102110006D2F0995DDCF88EC0E94E50E85FF14C078
:1021200060E288EC0E94D20E88EF0E94E50E807C6F
:10213000909112018917E1F180931201803409F125
:1021400050F4882379F1089580914E04811130C0B4
:1021500064E088EEE7CF803819F0803C09F10895FB
:1021600088ED0E94E50E90914E0481FD11C09230E1
:10217000F9F061EC88ED0E94D20E82E080934E046B
:10218000089588ED0E94E50E90914E0481FDEFCFF9
:10219000933071F063EC88ED0E94D20E83E0EECFB5
:1021A00081E0ECCF61EC88ED0E94D20E10924E04DB
:1021B0000895FC01848D089570E0685F7F4F660F7D
:1021C000771F860F971FFC015183408381E008959C
:1021D000482F80E1489F90011124205E310928306A
:1021E000310508F59091B1029923E9F0892F90E02B
:1021F000E3EBF2E061E070E02191243078F0322FDF
:1022000032953F7034130AC02F70DB0102C0AA0F51
:10221000BB1F2A95E2F79D018A2B932BB2E0E93B85
:10222000FB0751F7089590E080E0E2CFCF93DF9372
:10223000CDB7DEB728970FB6F894DEBF0FBECDBF7F
:10224000E22F29833A834B835C836D837E838F8364
:1022500098872091B1022E2B2093B102FE01339674
:10226000AE01475F5F4F2191243060F0A3EBB2E0F5
:1022700090E080E03D91311111C08F549D4FDC0101
:1022800012962C93E417F50771F728960FB6F89479
:10229000DEBF0FBECDBFDF91CF910895019686308E
:1022A000910541F7EFCFCF93DF93FC01DA018281F3
:1022B000882359F0813069F081E023813481232B18
:1022C00009F080E0DF91CF9108953483238381E08A
:1022D0008283838194810097B1F02D913C91119775
:1022E000232B51F3019794838383EB018881998198
:1022F0000196998388838D919C91119701971196EE
:102300009C938E93E6CF1282D7CF2F923F924F921B
:102310005F926F927F928F929F92AF92BF92CF9275
:10232000DF92EF92FF920F931F93CF93DF9300D032
:1023300000D0CDB7DEB76C017A8369835C834B83B1
:102340002C0182E1480E511C83E0282E5601A7E0A3
:10235000AA0EB11C12E0332433944601B0E18B0E77
:10236000911C3601EBE06E0E711C29813A8121151A
:10237000310509F4D4C0D60190968C918230F1F0E9
:10238000B0F5882309F45AC0813089F7AE014F5F58
:102390005F4FBE016D5F7F4FC5010E94340B8823E4
:1023A00009F4BDC0D6011596ED91FC911697808178
:1023B00091968C939197818192968C93F601568297
:1023C000458220A2D60192968C919297843011F486
:1023D00093961C92F60181A18250848325813681D7
:1023E000308727838287818784E080A305C083307C
:1023F00049F3843009F0BBCFD60192968C9184309A
:1024000039F1853009F44FC0823009F079C0AE014E
:102410004F5F5F4FBE016D5F7F4FC5010E94340B60
:10242000882309F47CC0F601858984A3D601169619
:102430009C928E92159790961C9297CFF6011483DA
:1024400085819681908787831287118730A29ECFDE
:10245000AE014F5F5F4FBE016D5F7F4FC5010E94B0
:10246000340B882309F45BC0D60155968C9155979F
:102470008330E1F656968C9156978130B9F698964E
:102480009C91989757968C91992351F0882371F2DB
:10249000F60133A2928996A3938997A385A3C6CF09
:1024A000813021F6F5CFAE014F5F5F4FBE016D5F0A
:1024B0007F4FC5010E94340B882389F1D601939682
:1024C0008C919397882309F4B1CF12968D919C91AA
:1024D000009709F4ABCFDC01ED91FC910190F08104
:1024E000E02D7401D60195960C91959797962C91B5
:1024F000979796964C91969794966C91099596CF4E
:10250000F60121A12250330BAE014F5F5F4FBE0198
:102510006D5F7F4FC3010E945311811187CF0F90D0
:102520000F900F900F90DF91CF911F910F91FF901F
:10253000EF90DF90CF90BF90AF909F908F907F9063
:102540006F905F904F903F902F9008952F923F9201
:102550004F925F926F927F928F929F92AF92BF92B3
:10256000CF92DF92EF92FF920F931F93CF93DF935F
:1025700000D000D0CDB7DEB76C017A8369835C836D
:102580004B832C0182E1480E511C83E0282E56011A
:10259000A7E0AA0EB11C12E0332433944601B0E147
:1025A0008B0E911C3601EBE06E0E711C29813A8175
:1025B0002115310509F4CFC0D60190968C91823057
:1025C000F1F0B0F5882309F45AC0813089F7AE01E3
:1025D0004F5F5F4FBE016D5F7F4FC5010E94340B9F
:1025E000882309F4B8C0D6011596ED91FC91169791
:1025F000808191968C939197818192968C93F6012C
:102600005682458220A2D60192968C919297843070
:1026100011F493961C92F60181A182508483258146
:102620003681308727838287818784E080A305C035
:10263000833049F3843009F0BBCFD60192968C9158
:10264000843039F1853009F44AC0823009F074C011
:10265000AE014F5F5F4FBE016D5F7F4FC5010E94AE
:10266000340B882309F477C0F601858984A3D60149
:1026700016969C928E92159790961C9297CFF60183
:10268000148385819681908787831287118730A272
:102690009ECFAE014F5F5F4FBE016D5F7F4FC501A3
:1026A0000E94340B882309F456C0D60155968C91AC
:1026B00055978330E1F698969C91989757968C9110
:1026C000992351F0882399F2F60133A2928996A3B7
:1026D000938997A385A3CBCF813049F6F5CFAE017F
:1026E0004F5F5F4FBE016D5F7F4FC5010E94340B8E
:1026F000882389F1D60193968C919397882309F4C6
:10270000B6CF12968D919C91009709F4B0CFDC0161
:10271000ED91FC910190F081E02D7401D601959628
:102720000C91959797962C91979796964C91969792
:1027300094966C9109959BCFF60121A12250330B01
:10274000AE014F5F5F4FBE016D5F7F4FC3010E94BF
:10275000531181118CCF0F900F900F900F90DF913C
:10276000CF911F910F91FF90EF90DF90CF90BF908E
:10277000AF909F908F907F906F905F904F903F9021
:102780002F90089580E00895089580E008952F9295
:102790003F924F925F926F927F928F929F92AF92F1
:1027A000BF92CF92DF92EF92FF920F931F93CF933E
:1027B000DF937B014A016901F901A080B180FB012F
:1027C0002180F90111821082FB01828160E181FD8B
:1027D00060E288EE0E94D20E3A2CA401F7016081DB
:1027E00080E00E94F60E582EF6E08F17B1F38111AB
:1027F0004EC088EC0E94E50E82FF5DC080E30E941F
:10280000E50E482E8A151B0411F008F0432CF60142
:10281000808191813501681A790A77FE02C0712C96
:10282000612CC42DD0E0C615D7050CF43E01562C02
:102830000E94AA0EF8E0FEBD0DB407FEFDCFF80120
:10284000552041F01EBC5A940DB407FEFDCF8EB545
:102850008193F6CF060D171D0E94AC0E64E088EC44
:102860000E94D20EF60180819181C80FD91FD183B9
:10287000C083421420F0CA15DB0508F4AECF88EF00
:102880000E94E50EF701928184FB91F99283852DD8
:10289000DF91CF911F910F91FF90EF90DF90CF903C
:1028A000BF90AF909F908F907F906F905F904F9070
:1028B0003F902F90089580EF582EE9CFAF92BF92AE
:1028C000CF92DF92EF92FF920F931F93CF93DF93FC
:1028D00000D000D0CDB7DEB77C01690158011C8261
:1028E0001B821A8219828E010F5F1F4F9E012D5F7E
:1028F0003F4F0E94560F811109C049815A816B8157
:102900007C8185019601C7010E94C7130F900F902B
:102910000F900F90DF91CF911F910F91FF90EF904B
:10292000DF90CF90BF90AF9008952F923F924F923B
:102930005F926F927F928F929F92AF92BF92CF924F
:10294000DF92EF92FF920F931F93CF93DF93CDB758
:10295000DEB765970FB6F894DEBF0FBECDBF3C0162
:10296000342E222E402EED8AEAA4FBA4188A1F865C
:102970001E861D868E01035F1F4F9E01215F3F4F04
:1029800040E00E94560F582E81111AC139822A82C6
:102990004B822D892C83DE82CD82B886AF82AE0138
:1029A0004F5F5F4F68E080E20E94AE0E4D855E850E
:1029B00060E080E10E94F60E811120C1E114F10473
:1029C00009F449C00F851889D80112968C91129785
:1029D00037FE47C0826012968C936501C114D10402
:1029E00009F411C19C2D8D2D8C149D0410F4982D8B
:1029F000892D9B878C874D855E856F8578898701BA
:102A00009E01255F3F4FC3010E94C713582EB6E0B9
:102A10008B1721F38111D4C0ECA5FDA53097A1F04F
:102A20006B857C850190F081E02D0190F081E02D97
:102A3000C5018C199D099A8789879E01275F3F4FA1
:102A4000A7018CA59DA509958B859C85C81AD90AD7
:102A50008815990518F64D855E8537FECBC080EA4E
:102A6000CAC0816012968C93129711966C908FEF6A
:102A7000860D803408F0C4C02D843E840E94970CDB
:102A80009B01AC0128573C4E4F4F5F4F298B3A8B2F
:102A90004B8B5C8BD80112968C9160E880FF60E4D0
:102AA00088EE0E94D20E512C712C8114910409F4ED
:102AB00076C063018614970408F46401CD8AA701E7
:102AC0006C2D80E10E94AE0E6C2D88E30E94D20E28
:102AD000F8016081606280EF0E94D20E88EC0E9453
:102AE000E50E87FFFBCF60E888EC0E94D20E88EFEE
:102AF0000E94E50E8F70582E412CB12CA12C552030
:102B000019F10E94970C29893A894B895C89621BCB
:102B1000730B840B950B97FF17C036E05316E9F043
:102B20004EE05416B1F054E0551209C08FEFA81AC8
:102B3000B80A2114310489F02A143B0471F460E0CE
:102B400088E30E94D20E2DC08C189D08EC0CFD1C51
:102B5000ACCF439493E0491691F360E088E30E9480
:102B6000D20ED7016C9180E10E94D20E6D8988E36C
:102B70000E94D20EF8016081606280EF0E94D20E46
:102B800088EC0E94E50E87FFFBCF60E888EC0E948E
:102B9000D20E88EF0E94E50E8F70582EB0CF5110E4
:102BA000CECF88EF0E94E50ED80112969C91129725
:102BB00085FB90F912969C934D855E855520D1F04A
:102BC000852D65960FB6F894DEBF0FBECDBFDF91A1
:102BD000CF911F910F91FF90EF90DF90CF90BF901A
:102BE000AF909F908F907F906F905F904F903F90AD
:102BF0002F90089580E860E00E94F60E582EE0CFF6
:102C00008AED582EDDCF4D855E85552009F427CFFE
:102C1000D7CF8F929F92AF92BF92CF92DF92EF92D7
:102C20000F93CF931F921F921F921F92912C812C72
:102C3000B12CA12CD12CC12CE12C062F25E040E099
:102C400060E00E949514C82F6CE271E080E090E093
:102C50000E94B60D0F900F900F900F908C2FCF9178
:102C60000F91EF90DF90CF90BF90AF909F908F909B
:102C700008958F929F92AF92BF92CF92DF92EF9280
:102C80000F931F921F923F932F934A015A01D12C09
:102C9000C12CEE24E39400E026E040E80E94951465
:102CA0000F900F900F900F900F91EF90DF90CF90BB
:102CB000BF90AF909F908F9008958F929F92AF9208
:102CC000BF92CF92DF92EF920F931F931F921F92AA
:102CD0001F930F934A015A01D12CC12C32E0E32EED
:102CE000022F26E040E80E9495140F900F900F905D
:102CF0000F901F910F91EF90DF90CF90BF90AF900A
:102D00009F908F9008955F926F927F928F929F9283
:102D1000AF92BF92CF92DF92EF92FF920F931F93E9
:102D2000CF93DF93CDB7DEB7C054D1090FB6F89477
:102D3000DEBF0FBECDBF3C01F62E542EE22E932EE9
:102D4000CE0101966C018C01242F49E050E0C301B3
:102D50000E945D16811118C0AB80BC809F92EF92DB
:102D6000DF92CF9280E4882E912CD12CC12C92E05E
:102D7000E92E052D26E040E86F2DC3010E94951431
:102D80000F900F900F900F90C05CDF4F0FB6F8942C
:102D9000DEBF0FBECDBFDF91CF911F910F91FF908E
:102DA000EF90DF90CF90BF90AF909F908F907F90EB
:102DB0006F905F9008958F929F92AF92BF92CF9243
:102DC000DF92EF920F93C42ED12C1F921F921F926D
:102DD0001F92912C812CB12CA12CE12C062F21E0EB
:102DE00043E2FC016285828193810E9495140F90D9
:102DF0000F900F900F900F91EF90DF90CF90BF90BA
:102E0000AF909F908F9008958F929F92AF92BF92B4
:102E1000CF92DF92EF920F93C62ED12C1F921F926A
:102E20005F934F9324E0822E912C34E0A32EB12C9B
:102E3000E12C00E020E043EAFC016285828193817D
:102E40000E9495140F900F900F900F900F91EF909C
:102E5000DF90CF90BF90AF909F908F9008958F920A
:102E60009F92AF92BF92CF92DF92EF920F93C42EB8
:102E7000D12C1F921F921F921F92912C812CB12C4A
:102E8000A12CE12C062F23E043E2FC016285828124
:102E900093810E9495140F900F900F900F900F91B7
:102EA000EF90DF90CF90BF90AF909F908F9008955C
:102EB000CF92DF92FF920F931F93CF93DF9300D0B7
:102EC00000D0CDB7DEB78C01F62E19821A821B8294
:102ED0001C82462F61E10E94DB164F2D60E1C80184
:102EE0000E94DB164F2D64E0C8010E942F1783E07B
:102EF000C82ED12CAE014F5F5F4F6F2DC8010E94CD
:102F00000417811114C089819A81AB81BC819D7F96
:102F100083309140A041B10551F064E670E080E05B
:102F200090E00E94B60D81E0C81AD10819F74F2D24
:102F300064E1C8010E94DB164F2D60E1C8010E94C8
:102F4000DB1664E170E080E090E00E94B60D0F9027
:102F50000F900F900F90DF91CF911F910F91FF90E5
:102F6000DF90CF9008952F923F924F925F926F9291
:102F70007F928F929F92AF92BF92CF92DF92EF9209
:102F8000FF920F931F93CF93DF93CDB7DEB7E897F0
:102F90000FB6F894DEBF0FBECDBFDC011A963C9190
:102FA000311125C1922E242E362E3C01FC01E280E7
:102FB000F380D701ED91FC910190F081E02D60E06C
:102FC000C70109958C01009709F414C1FC01C08068
:102FD000D180C114D10409F410C15301F4E0AF0E43
:102FE000B11CDC011196BC92AE9214969C92FE012B
:102FF00031962F019F0148E050E060E0D301129626
:103000008D919C910E943916982EF801148281119D
:10301000FAC08D8191ED992E893059F58980D701BB
:10302000ED91FC910280F381E02D222D41E0632D92
:10303000C7010995F3018287882309F4E1C09885C7
:103040009583682F828193810E940916982ED8015A
:10305000CD92DC92882339F1D701ED91FC91048067
:10306000F581E02DD3011A966C91C7010995F30102
:103070001286892DE8960FB6F894DEBF0FBECDBF3D
:10308000DF91CF911F910F91FF90EF90DF90CF9044
:10309000BF90AF909F908F907F906F905F904F9078
:1030A0003F902F900895811082C0950142E0F30176
:1030B0006285828193810E94790C982E8111D9CFEB
:1030C0001F921F925F924F9258E0852E912C68E0DC
:1030D000A62EB12CD12CC12C79E2E72E00E026E0FF
:1030E00040EAF3016285828193810E949514982EB3
:1030F0000F900F900F900F908111BBCF8B81D30158
:103100001B968C931B97820120E048E050E01A96B2
:103110006C911A9712968D919C910E945D16982E33
:103120008111A7CF4B815C8120E0F3016285828110
:1031300093810E945D16982E81119BCF498150E0AA
:103140008E010F5D1F4F20E0D3011A966C911A97E4
:1031500012968D919C910E945D16982E811189CFB7
:103160001F921F921F921F92912C812CB12CA12C87
:10317000E12C0E8129E040E0F30162858281938198
:103180000E949514982E0F900F900F900F90811120
:1031900070CF11E0D3011B968C911B978117D0F053
:1031A000412F68E0C3010E942F171F5FF3CF482D06
:1031B000413208F040E250E09201D3011A966C913E
:1031C0001A9712968D919C910E943916982E811112
:1031D00050CF6BCF1296ED91FC911397EA58FF4FA9
:1031E00080818460808381E050968C9342CF49ED4A
:1031F000942E3FCF36ED932E3CCF27ED922E39CF34
:1032000084ED982E36CFD182C08233CF2F923F9259
:103210004F925F926F927F928F929F92AF92BF92E6
:10322000CF92DF92EF92FF920F931F93CF93DF9392
:10323000CDB7DEB7CB57D1090FB6F894DEBF0FBEBE
:10324000CDBFDC0116963C91311106C2522E342EB0
:10325000462E3C01FC01A480B580158ED501ED9170
:10326000FC910190F081E02D60E0C50109956C01B1
:103270000097E9F4A6ED3A2E832DC558DF4F0FB61F
:10328000F894DEBF0FBECDBFDF91CF911F910F919C
:10329000FF90EF90DF90CF90BF90AF909F908F9076
:1032A0007F906F905F904F903F902F900895FC011A
:1032B000808091808114910409F4D1C18301095F58
:1032C0001F4F1183008354829E0126593F4F48E0CF
:1032D00050E060E0D30114968D919C910E943916C4
:1032E000E82E8111C2C1AB96FFACAB97F60191827B
:1032F0008082D501ED91FC910280F381E02D232D98
:1033000040E0642DC5010995F3018683882309F403
:10331000A9C1E2969FADE2979087682F848195813D
:103320000E940916382ED501ED91FC91D601149614
:103330001C92882359F00480F581E02DD301169664
:103340006C91C5010995F301168296CF0190F08129
:10335000E02DD30116966C91C5010995009709F4EB
:1033600089CFFC015482980141E0D30116966C91FB
:10337000169714968D919C910E94790CF11085C03E
:10338000EC962FACEC975301B2E0AB0EB11C70E29F
:10339000472E71E0572EE1E4EE2EF12CEC0EFD1ECF
:1033A000E0E1EE0EF11CF6E28F2EF1E09F2E6E01B1
:1033B000F1E1CF0ED11C231409F41DC123965FAE99
:1033C0004EAE23972596BFAEAEAE259726961FAE7E
:1033D00026972B961FAE2B972C961FAE2C972F96C9
:1033E0001FAE2F9761961FAE1EAE6197A2961FAEBD
:1033F000A297A3961FAEA397A4961FAEA497AA96D2
:103400001FAEAA972896FFAEEEAE28972A96FFAE7B
:10341000EEAE2A972E96FFAEEEAE2E979E012F5B54
:103420003F4F432DF3016681848195810E9483166D
:10343000D30157968C915797823008F0DCC09A825E
:103440008982BC82AB821D821A861B861E86188AE0
:103450001F8619A21AA21BA219A6DF82CE82D986C4
:10346000C886DD86CC869E012F5F3F4F432D169682
:103470006C91169714968D919C910E948316F3017E
:103480008789823008F5339496CF4F2D433108F069
:1034900042E150E09E0126593F4FD30116966C91B0
:1034A000169714968D919C910E943916E82E8823C8
:1034B00009F466CFD301ED91FC910480F581E02DF4
:1034C000C30109953E2CD8CEF12CD30157964C91CF
:1034D000579731EDE32E423068F3980116966C91C0
:1034E000169714968D919C910E94790C68EE73E06A
:1034F00080E090E00E94B60D1F921F921F921F92D3
:10350000912C812CB12CA12CD12CC12CE12CF301BC
:10351000048929E040E06681848195810E949514A8
:10352000E82E0F900F900F900F908111C3CF68EE8F
:1035300073E080E090E00E94B60D10E01E01F1E41F
:103540002F0E311C412E512CD30157968C91579739
:103550008150990B481659060CF079C0460C571C3F
:10356000F1104CC0F201C288D12C1F921F921F9201
:103570001F92912C812CB12CA12CE12C00E02AE08F
:1035800041E2D30116966C91169714968D919C91F9
:103590000E9495140F900F900F900F90811153C0BF
:1035A0008CE291E0F10191838083D2015296CC901C
:1035B000D12C3F922F92E1E0F0E0EC0FFD1FFF9342
:1035C000EF9340E4842E912C50E8A52EB12C62E2BA
:1035D000E62E00E026E041E8D30116966C9116979E
:1035E00014968D919C910E9495141F5F0F900F90DF
:1035F0000F900F90A7CFFF24F39467CFF201C288FA
:10360000D12C1F921F921F921F92912C812CB12CB2
:10361000A12CE12C5E960C915E972BE041E2169670
:103620006C91169714968D919C910E9495140F9011
:103630000F900F900F90882309F494CF853009F4F0
:1036400091CFE82E37CF853009F4AACFFACF81E0A9
:10365000F301848F312C10CE29ED322E0DCE97ED53
:10366000392E0ACE84ED382E07CEF6019182808263
:1036700021CF3F924F925F926F927F928F929F9253
:10368000AF92BF92CF92DF92EF92FF920F931F9370
:10369000CF93DF93EC01F62E372E2C0182E1480EFA
:1036A000511C712C612C10E08F898150990B681688
:1036B00079060CF5F201C1902F01D12C1F921F92B7
:1036C0003F92FF9288248394912CAA24A394B12C36
:1036D00022E0E22E00E029E041E26E818C819D81B2
:1036E0000E949514182BFFEF6F1A7F0A0F900F900E
:1036F0000F900F90D9CF812FDF91CF911F910F9114
:10370000FF90EF90DF90CF90BF90AF909F908F9001
:103710007F906F905F904F903F900895CF93DF938D
:103720001F92CDB7DEB7898380916B05882339F06E
:10373000BE016F5F7F4F8FE495E00E94391B80913F
:103740004C05882339F0BE016F5F7F4F80E395E021
:103750000E94391B80912D05882339F0BE016F5FCF
:103760007F4F81E195E00E94391B80910E058823EF
:1037700039F0BE016F5F7F4F82EF94E00E94391BEA
:103780000F90DF91CF9108952F923F924F925F92C9
:103790006F927F928F929F92AF92BF92CF92DF9261
:1037A000EF92FF920F931F93CF93DF93CDB7DEB7C6
:1037B00068970FB6F894DEBF0FBECDBF1B8A38E006
:1037C0003C8B3CE33D8B8A3F3FEF9307D9F416EDEA
:1037D000812F68960FB6F894DEBF0FBECDBFDF9184
:1037E000CF911F910F91FF90EF90DF90CF90BF90FE
:1037F000AF909F908F907F906F905F904F903F9091
:103800002F900895222E642E362E7C01DC01169610
:103810000D911C911797CE01439617969C938E930A
:1038200016971A962C939E012F5F3F4F42E150E06E
:1038300060E0C7010E943916782EF70117830683CE
:10384000182F8111C5CF49845A848B849C84FD81B3
:10385000FF8B3E81388F670186E5C80ED11C56016B
:103860001E8AD5018D919D915D010097D1F5BE898C
:10387000BF5FBE8BB031A9F7F601819191916F01C5
:10388000009709F06EC07394F0E17F12F5CFF70155
:103890008681978117ED892B09F49ACF2286262DF0
:1038A00040E0632DC7010E940D0C082F14ED882302
:1038B00009F48ECF682FC7010E94620C009709F4AB
:1038C00086CFDC0114962C92602FC7010E94091646
:1038D000182F882309F47CCF602FC7010E94EB0BBF
:1038E00077CFDC01ED91FC910084F185E02D099505
:1038F0008111BDCFF501929182918F01DC01ED9193
:10390000FC910088F189E02D688D0995882309F4E0
:10391000AECFF80180819181DC01ED91FC910484AE
:10392000F585E02DA401B2010995882361F0022DEF
:10393000262D432D6E89C7010E94BE0F182F813D91
:1039400009F495CF45CFF80180819181DC01ED919B
:10395000FC910684F785E02D6F8909958111E7CFE9
:1039600086CFDC01ED91FC910084F185E02D099575
:10397000811189CFF601929182918F01DC01ED9145
:10398000FC910088F189E02D688D099581110DC0A9
:10399000022D262D432D672DC7010E94BE0F182F23
:1039A000877F813D09F014CF6ECFF801808191812E
:1039B000DC01ED91FC910484F585E02DA401B201B8
:1039C0000995811160CFF80180819181DC01ED9131
:1039D000FC910684F785E02D6F8909958823C1F253
:1039E00052CFCF92DF92EF92FF921F93CF93DF934C
:1039F000EC01162F7A01FA0180819181A281B381B5
:103A00008130F3E09F07F1E0AF07B105C9F170F431
:103A10008115E1E09E07AE07B10509F450C0813081
:103A20009140A140B10561F180E041C0833021E0C7
:103A3000920720E1A207B10529F083309340A0410D
:103A4000B10591F7412F64E1CE010E94DB16412FB1
:103A500060E1CE010E94DB1664E170E080E090E05E
:103A60000E94B60D6A85F701218126952170677045
:103A7000412F8A819B810E94C41B1092B902D4CF2E
:103A80008091B9028111D0CF412F61E1CE010E9416
:103A9000DB16412F60E1CE010E94DB16412F64E06E
:103AA000CE010E942F1781E08093B90281EBDF9154
:103AB000CF911F91FF90EF90DF90CF900895462F08
:103AC00061E1CE010E94DB16412F60E1CE010E9430
:103AD000DB161092B9028A8587701770880F880FDD
:103AE000880F182B09F4A0CFEA80FB806701F6E568
:103AF000CF0ED11CD0E0C0E0D6018D919D916D011B
:103B00000097C1F0DC01ED91FC910084F185E02D7E
:103B1000099518130FC0AB96CC0FDD1FCE0DDF1D1E
:103B200088819981DC01ED91FC910480F581E02D83
:103B300009957ACF2196C031D105F1F675CFCF9294
:103B4000DF92EF92FF920F931F93CF93DF93CDB746
:103B5000DEB72E970FB6F894DEBF0FBECDBFFC01C7
:103B60002089211111C010E0812F2E960FB6F894F4
:103B7000DEBF0FBECDBFDF91CF911F910F91FF90A0
:103B8000EF90DF90CF9008957C010E94970CF70191
:103B90000485158526853785601B710B820B930B79
:103BA00097FDE1CF81E090E09E878D878E010F5FCA
:103BB0001F4F9E01235F3F4F41E0628582819381C9
:103BC0000E945E14182F811121C082E0D82E01E0DE
:103BD00089818D2139F119861A861B861C86AE01D2
:103BE000475F5F4F602FC7010E940417C82E8111E5
:103BF00019C0AE01475F5F4F602FC7010E94F11CE3
:103C0000813B19F0882371F0C82E1C2D0E94970C5F
:103C10006C597F4F8F4F9F4FF70164877587868759
:103C20009787A2CFDD0C0F5F083091F601E0F70116
:103C30008385801758F319861A861B861C86AE0169
:103C4000475F5F4F602FC7010E940417D82E811174
:103C500017C089859A85877091708130914081F471
:103C60008B859C8581609C878B87AE01475F5F4F0A
:103C7000602FC7010E94F11C813B29F0811102C015
:103C80000F5FD5CFD82E1D2DC1CFCF938091440487
:103C900083FF7EC08EE094E00E947B028091490405
:103CA0001F928F9389E094E09F938F930E94140357
:103CB00087E094E00E947B0280914A04282F082E1E
:103CC000000C330B3F938F9384E094E09F938F938A
:103CD0000E94140382E094E00E947B0280914B04D6
:103CE000282F082E000C330B3F938F938FEF93E018
:103CF0009F938F930E9414038DEF93E00E947B02A9
:103D000080914C04282F082E000C330B3F938F9387
:103D10008AEF93E09F938F930E94140388EF93E0C0
:103D20000E947B0280914D04282F082E000C330B3B
:103D30003F938F9385EF93E09F938F930E9414039B
:103D400082EF93E00E947B02809143041F928F9345
:103D50008FEE93E09F938F930E9414038DEE93E078
:103D60000E947B02809142041F928F938AEE93E01F
:103D70009F938F930E94140387EE93E00E947B022F
:103D80008DB79EB74C960FB6F8949EBF0FBE8DBFF1
:103D9000E0914504F0914604309751F0C0914904F8
:103DA0000480F581E02D89E494E00995C0934904ED
:103DB0000E94B60C9093480480934704CF910895D5
:103DC00010923B04ECE9F2E0118212821382148219
:103DD0001582168217820E94CD0485E0E9E4F4E0A2
:103DE000DF011D928A95E9F7109243041092420474
:103DF0000E94451E90E080E00E94630690E080E013
:103E00000C944D06AF92BF92CF92DF92EF92FF9249
:103E10000F931F93CF936091F0047091F104409140
:103E2000E4045091E5042091D8043091D9048091A4
:103E3000CC049091CD04E091AF02F091B0026E17E6
:103E40007F07B1F4E091AD02F091AE02E417F507FF
:103E500079F4E091AB02F091AC02E217F30741F480
:103E6000E091A902F091AA02E817F90709F45FC0EE
:103E70007093B0026093AF025093AE024093AD02D4
:103E80003093AC022093AB029093AA028093A902D4
:103E900088E0E1EBF2E0DF011D928A95E9F72091DD
:103EA000E8043091E9044091EA045091EB046091F8
:103EB000EC047091ED048091EE049091EF040E9467
:103EC00016112091DC043091DD044091DE04509104
:103ED000DF046091E0047091E1048091E20490912C
:103EE000E3040E9416112091D0043091D104409136
:103EF000D2045091D3046091D4047091D504809180
:103F0000D6049091D7040E9416112091C4043091D8
:103F1000C5044091C6045091C7046091C8047091D3
:103F2000C9048091CA049091CB040E9416110E948A
:103F3000B60C7C010E948B1080914E04813009F4F4
:103F40005DC008F45FC0823029F0833009F462C09C
:103F5000C0E017C0C0E080919F04807F803189F469
:103F60000E94970C68537F4F8F4F9F4F6093A4021E
:103F70007093A5028093A6029093A70280E280939B
:103F80009F0484ECC82E85E0D82E94EEA92E95E0EF
:103F9000B92E8601F801819191918F01009739F036
:103FA000DC01ED91FC910680F781E02D0995A016CA
:103FB000B10681F780919F04803409F4B7C060F5A1
:103FC000803209F49DC0803309F4AAC0813161F5C3
:103FD0001092E405F601819191916F01009739F0FB
:103FE000DC01ED91FC910480F581E02D0995C0166E
:103FF000D10681F782E180939F0416C083E180930C
:104000009F04A6CF80919F04807F803109F4A0CFC8
:1040100081E1F5CFC1E09FCF813509F4B1C008F04F
:1040200059C0803509F495C02FB7F89480913D04AC
:1040300090913E04A0913F04B09140042FBF8E198F
:104040009F098536910560F09F938F9389EA91E0EF
:104050009F938F930E9414030F900F900F900F90D7
:1040600080919F049091A802981749F18093A8022B
:104070001F928F9388E991E09F938F930E9414037E
:104080000F900F900F900F908091A8028039B9F493
:1040900080914E04823009F096C083E191E09F93B5
:1040A0008F938DE891E09F938F930E9414030E9459
:1040B00079060E948E1B0F900F900F900F9081E059
:1040C000CF911F910F91FF90EF90DF90CF90BF9015
:1040D000AF900895803809F466C0803A09F0A4CF03
:1040E0000E94970C68537F4F8F4F9F4F6093A4029D
:1040F0007093A5028093A6029093A70280E27BCFE3
:104100000E94970C0091A4021091A5022091A60292
:104110003091A702601B710B820B930B97FD84CF2C
:1041200061E088EE0E94D20E80E465CF88EE0E94A6
:10413000E50E80FD79CF60E488EC0E94D20E88ED18
:104140000E94E50E682F686088ED0E94D20E80E51F
:1041500052CF88EC0E94E50E86FF66CF81E5809302
:104160009F040E94970C6C507E4F8F4F9F4F60931F
:10417000A4027093A5028093A6029093A70254CF45
:104180000E94970C0091A4021091A5022091A60212
:104190003091A702601B710B820B930B97FD44CFEC
:1041A00080E880939F042C2F40E060E08EE695E04D
:1041B0000E94C41B882329F0823D09F435CF80EA90
:1041C0001ACF80E918CF88E191E069CFCF93DF93D0
:1041D000882309F45DC09EE7980F933020F5C2E074
:1041E000D9E3823831F0C4E0D7E4833811F4C1E078
:1041F000D3E50E9479068C2309F44AC08D2F0E94D2
:10420000B4040E94CD042FEF41EE54E02150404011
:104210005040E1F700C000008D2F0E94A804DF91FC
:10422000CF910C94CD049CEF980F913AB0F390E2AB
:10423000980F983088F4877021E030E0A90102C01F
:10424000440F551F8A95E2F7CA01809590913C046E
:10425000892380933C04E3CF9BE5980F933030F49F
:1042600090E080E0DF91CF910C94630698E5980F81
:10427000973130F490E080E0DF91CF910C944D06BF
:10428000803F30F00E945703DF91CF910C94451E80
:10429000DF91CF910895CF93DF93882309F402C172
:1042A0009EE7980F933020F5C2E0D9E3823831F0D1
:1042B000C4E0D7E4833811F4C1E0D3E50E94790665
:1042C0008C2309F0EFC08D2F0E94B4040E94CD040E
:1042D0002FEF81EE94E0215080409040E1F700C044
:1042E00000008D2F0E94A804DF91CF910C94CD0483
:1042F0009CEF980F913A18F40E94B404F5CF90E225
:10430000980F983068F4877021E030E001C0220FE8
:104310008A95EAF780913C04822B80933C04E4CF99
:104320009BE5980F933080F4853A41F0863A49F046
:1043300083E890E0DF91CF910C94630681E890E0F0
:10434000F9CF82E890E0F6CF98E5980F973108F022
:1043500090C0883A09F448C0893A09F448C08A3ABA
:1043600009F448C08B3A09F448C08C3A09F448C0B3
:104370008D3A09F448C08E3A09F448C08F3A09F4DE
:1043800048C0813B09F448C0803B09F448C0823BE7
:1043900009F448C0833B09F448C0843B09F448C091
:1043A000853B09F448C0863B09F448C0873B09F4C3
:1043B00048C0883B09F448C0893B09F448C08A3B9F
:1043C00009F448C08B3B09F448C08C3B09F448C051
:1043D0008D3B09F448C08E3B09F448C090E080E072
:1043E000DF91CF910C944D0682EE90E0F9CF89EEEB
:1043F00090E0F6CF8AEE90E0F3CF85EB90E0F0CF3F
:1044000086EB90E0EDCF83EB90E0EACF84EB90E099
:10441000E7CF87EB90E0E4CF8CEC90E0E1CF8DEC40
:1044200090E0DECF83E891E0DBCF8AE891E0D8CF5F
:1044300082E991E0D5CF84E991E0D2CF81E292E0A8
:10444000CFCF83E292E0CCCF84E292E0C9CF85E285
:1044500092E0C6CF86E292E0C3CF87E292E0C0CF7F
:104460008AE292E0BDCF8FE690E0BACF80E790E09D
:10447000B7CF8F3B79F410923C040E94E01E2FEFDF
:1044800080E792E0215080409040E1F700C00000BA
:104490000E94A406803F30F00E941D04DF91CF915E
:1044A0000C94451EDF91CF910895CF92DF92EF9249
:1044B000FF920F931F93CF93DF9300D000D01F92F2
:1044C000CDB7DEB76C0185E0F601DE0111960190F3
:1044D0000D928A95E1F7F601408151812381348163
:1044E00091E02115310531F05F3F19F491E04F3F24
:1044F00009F090E090FD99C0F6010281F580F294F8
:104500009FE0F92249835A830B83722F3D832C83CA
:10451000602F8D810E94F504182FE92FE295EF702E
:10452000EF3008F082C0F0E0E856FD4D0C94F42F17
:10453000A722A722E522E5225B238D23152315233D
:10454000A323152379247924152315233525F92F41
:10455000FF70FF2E907F19F0F29480EFF822002375
:10456000C9F0FF2039F080913B04F82AF0923B0417
:104570000E94CD04812F0F900F900F900F900F90FD
:10458000DF91CF911F910F91FF90EF90DF90CF902F
:104590000C944B21812F0E94E620FF2009F445C096
:1045A000F09480913B04F822F0923B040F900F901E
:1045B0000F900F900F90DF91CF911F910F91FF906F
:1045C000EF90DF90CF900C94CD04892F8F70907F67
:1045D000903211F08295807F112379F0113009F427
:1045E00049C0002309F455C0FF2059F0F601958118
:1045F00090FF8DC19F70958304C0002321F1F110BD
:104600000FC00F900F900F900F900F90DF91CF91F0
:104610001F910F91FF90EF90DF90CF900C94430685
:1046200021E0F212EECF80933A040F900F900F909A
:104630000F900F90DF91CF911F910F91FF90EF900E
:10464000DF90CF900895F11011C010923A040F90AE
:104650000F900F900F900F90DF91CF911F910F91BE
:10466000FF90EF90DF90CF900C94380691E0F91214
:10467000ECCFDBCF002349F0E5E0EF15B0F29091ED
:104680003C04982309F4BDCFE2CFF4E0FF1568F2B3
:10469000DECFFF20E1F2812F0F900F900F900F904F
:1046A0000F90DF91CF911F910F91FF90EF90DF90CE
:1046B000CF900C94E620892F869586958370C1F063
:1046C000813009F0B2CF812F9370011102C090E0C8
:1046D00080E00F900F900F900F900F90DF91CF918F
:1046E0001F910F91FF90EF90DF90CF900C944D06AB
:1046F000812F9370011102C090E080E00F900F9025
:104700000F900F900F90DF91CF911F910F91FF901D
:10471000EF90DF90CF900C946306002389F00E9405
:104720001D040F900F900F900F900F90DF91CF917D
:104730001F910F91FF90EF90DF90CF900C94451E4A
:104740000E945703EECF892F837009F064C00111D6
:104750006CCF812F829586958770880F880F412FA7
:104760004F70C42ED12CF12CE12C082E04C0CC0C9F
:10477000DD1CEE1CFF1C0A94D2F740E050E0BA01A9
:1047800014FF11C00FE010E020E030E004C0000F83
:10479000111F221F331F8A95D2F7B901A801409536
:1047A00050956095709500913203109133032091DC
:1047B0003403309135039695969593709230E9F0D5
:1047C00028F5913089F04C295D296E297F294023F5
:1047D0005123622373234093320350933303609336
:1047E00034037093350321CFC02AD12AE22AF32A59
:1047F0004C295D296E297F29EECF4C295D296E2930
:104800007F294027512762277327E5CF4023512373
:1048100062237323EDCF8695002311F0892F8170D9
:10482000882309F402CF812F829586958770880F9F
:10483000880F412F4F70C42ED12CF12CE12C082E63
:1048400004C0CC0CDD1CEE1CFF1C0A94D2F740E027
:1048500050E0BA0114FF11C00FE010E020E030E09A
:1048600004C0000F111F221F331F8A95D2F7B90110
:10487000A801409550956095709500913603109170
:1048800037032091380330913903969596959370AC
:104890009230E9F028F5913089F04C295D296E2994
:1048A0007F2940235123622373234093360350937F
:1048B00037036093380370933903B7CE0C291D2951
:1048C0002E293F29402B512B622B732BEECF4C29E5
:1048D0005D296E297F294027512762277327E5CF5D
:1048E00040235123622373234C295D296E297F299C
:1048F000DCCF803F09F44EC0D0F480E4810F8032D9
:1049000070F1002309F4ACC0FF2009F4A6C0812F88
:104910000E944B21193309F099C0FFEF21EE84E08A
:10492000F15020408040E1F700C000007ECE823F81
:1049300009F470C008F45BC0833F19F7002309F441
:104940007CC0292F2F7181E090E0A0E0B0E004C08E
:10495000880F991FAA1FBB1F2A95D2F73AC0E12FD3
:10496000E071FE2E892F8F71002351F00E94C20545
:10497000812F8295807FF11044CE812F8F7041CEA0
:104980000E949E05812F8295807FF11060CE812F3D
:104990008F705DCE002331F1F4E0FF1508F445CEB1
:1049A000292F2F7181E090E0A0E0B0E004C0880FD3
:1049B000991FAA1FBB1F2A95D2F740913603509129
:1049C0003703609138037091390384279527A62710
:1049D000B7278093360390933703A0933803B0939F
:1049E000390323CE25E02F1508F41FCED9CF892F08
:1049F0008F71002399F00F900F900F900F900F90F0
:104A0000DF91CF911F910F91FF90EF90DF90CF90AA
:104A10000C94C205892F8F71002369F30F900F90BA
:104A20000F900F900F90DF91CF911F910F91FF90FA
:104A3000EF90DF90CF900C949E0510923603109269
:104A400037031092380310923903EFCD133509F470
:104A500064CF173409F0E9CD60CF892F8F71CBCFA8
:104A6000F11019CE892F8F71D9CF8111DECD00239E
:104A700009F4DBCD10923C040E94E01E8FEF90E71A
:104A8000E2E081509040E040E1F700C000000E9469
:104A9000A4060F931F93CF93DF938091FF02807F33
:104AA000B9F48091FC02882399F080913103109130
:104AB00000036091FA027091FB02C091FD02D09157
:104AC000FE0221E06F3F09F020E006E0181305C068
:104AD000DF91CF911F910F91089531E0209721F040
:104AE000322F7F3F09F030E090E030FD33C0089F67
:104AF000F001099FF00D1124DF01AF5FBC4F11964B
:104B00003C911197371326C03C91361323C012965F
:104B10003C91129731111EC013964D915C914C1B24
:104B20005D0B483C5105B0F48091FF028F708061AD
:104B30008093FF02EA5FFC4F80818F7080618083E9
:104B40008AEF92E00E945522DF91CF911F910F9141
:104B50000C94E20501968770B9CF9F92AF92BF92F5
:104B6000CF92DF92EF92FF920F931F93CF93DF9339
:104B7000CDB7DEB761970FB6F894DEBF0FBECDBFDD
:104B80008C0185E0F801DE011D9601900D928A9559
:104B9000E1F7F80140815181F280C380D480909187
:104BA000FA026091FB022091FD023091FE0281E049
:104BB0002115310531F06F3F19F481E09F3F09F075
:104BC00080E0F82FF1709F2E80FD49C18AEFA82E5A
:104BD00082E0B82EE090FC02F601E21BF30BEE201F
:104BE00009F400C18091FF02782F707FE83CF10545
:104BF00008F0BAC0711181C0EF2C651322C0941364
:104C000020C0F1101EC08F7080618093FF02C5012B
:104C10000E9455228091FF02F80185838E2D6196B6
:104C20000FB6F894DEBF0FBECDBFDF91CF911F91BD
:104C30000F91FF90EF90DF90CF90BF90AF909F903B
:104C4000089581E0C114D10431F05F3F19F481E08F
:104C50004F3F09F080E080FD24C081E08F25F82FD0
:104C6000F170BF2E80FF3FC080913103209100037F
:104C700036E0821318C07C2DD98AC88A6F2D8989A5
:104C80000E94F504292F22952F70223000F1243044
:104C900028F59F7001F1F8019581907FE1F4E92CEE
:104CA000BDCF80E0DCCF90E0389FF001399FF00D60
:104CB0001124EF5FFC4F6181561306C060814613DB
:104CC00003C062816F110FC001968770D2CF9F70B1
:104CD00011F0882321F3805E883008F3C8010E9418
:104CE00055229B2CDCCFFF2009F498CF8091FF0246
:104CF00081608093FF02E12C91CF651306C094136D
:104D000004C0F801FF2009F488C04D875E87FF8644
:104D10007C2DD98AC88A6F2D89890E94EC05882349
:104D200009F4ABC0FF2009F4A8C08091FF028032D3
:104D300070F02091FA023091FB0238872F83198698
:104D4000DB86CA868C87CE0107960E94552286E0B4
:104D5000F801AAEFB2E001900D928A95E1F70E9466
:104D60004925EE24E3945ACF71110AC08AEF92E0EC
:104D70000E94552286E0F50111928A95E9F7BBCF92
:104D800065130FC094130DC0F1100BC0F80185839B
:104D9000C8010E94552286E0F50111928A95E9F733
:104DA0003DCF4D875E87FF867C2DD98AC88A6F2DBF
:104DB00089890E94EC05882309F45FC0FF2009F46B
:104DC0005CC08091FF02803210F22091FA02309193
:104DD000FB023A8329831B82DD82CC828E83CE0143
:104DE0000196B3CFE83CF105B0F6EF2CFF2009F4B3
:104DF00044C065131FC094131DC08091FF0280FD45
:104E000010C0982F907F69F0F8018583903F31F0B2
:104E1000982F907F905F8F70892B8583C8010E94A7
:104E2000552286E0F801AAEFB2E001900D928A9532
:104E3000E1F7F4CE4D875E87FF867C2DD98AC88A3C
:104E40006F2D89890E94EC05811181CF8091FF022D
:104E500081608093FF02C8010E945522DFCEFF20AF
:104E600061F04D875E87FF867C2DD98AC88A6F2DB9
:104E700089890E94EC0581116ACFC8010E945522E0
:104E800070CF1F93CF93DF93CDB7DEB767970FB681
:104E9000F894DEBF0FBECDBF4B8B5C8B6D8B7E8BD2
:104EA0008F8B1A8A198A85E0FE017396DE011D96A2
:104EB00001900D928A95E1F786E0FE013D96DE01B4
:104EC000179601900D928A95E1F7CE0107960E9400
:104ED000AD25811137C086E0FE013796DE011196BF
:104EE00001900D928A95E1F79F8188852A853B85FF
:104EF000232B39F08F3F19F481E09F3F19F080E0B8
:104F000001C081E080FD1EC02091000330E0C90196
:104F1000019687709927409131034817190659F176
:104F200096E0929FD001939FB00D1124AF5FBC4FCC
:104F3000FE01319601900D929A95E1F7809300035E
:104F40000E94E20516E080913103909100038917D9
:104F500009F1819FC00111248F5F9C4F0E94AD25F4
:104F60008823C1F08091310390E0019687709927E2
:104F700080933103E8CF10923C040E94E01E10920F
:104F800000031092310386E0EAEFF2E0DF011D92A8
:104F90008A95E9F767960FB6F894DEBF0FBECDBFCE
:104FA000DF91CF911F910895CF93DF9300D01F928F
:104FB000CDB7DEB72091F502243041F520911001E4
:104FC000222321F123E029839B838A8382E080933B
:104FD000E9008FEF9091E800815095FD06C095EDB6
:104FE0009A95F1F700008111F5CF8091E80085FFD7
:104FF0000DC050E040E063E070E0CE0101960E94F9
:10500000A40A8091E8008E778093E8000F900F90BB
:105010000F90DF91CF910895CF93DF9300D01F922F
:10502000CDB7DEB72091F502243081F52091100133
:10503000222361F119821A821B8222E0298381389E
:10504000910520F0805891099B838A8382E08093A8
:10505000E9008FEF9091E800815095FD06C095ED35
:105060009A95F1F700008111F5CF8091E80085FF56
:105070000DC050E040E063E070E0CE0101960E9478
:10508000A40A8091E8008E778093E8000F900F903B
:105090000F90DF91CF9108952091F502243049F5CA
:1050A00022E02093E9002FEF3091E800215035FDF8
:1050B00006C035ED3A95F1F700002111F5CF2091AA
:1050C000E80025FF16C02091100150E040E063E0A9
:1050D00070E0222339F021E02093F10050E040E01D
:1050E00065E070E00E94A40A8091E8008E778093CA
:1050F000E8000895CF93DF932091F502243011F555
:1051000021E02093E90021E8215021F03091E800CE
:1051100035FF1BC02091E80025FF14C0EC0150E0D2
:1051200040E068E070E00E94A40A8091E8008E7779
:105130008093E80088E0FE01A2EEB2E001900D92BB
:105140008A95E1F7DF91CF910895EFE3F1E0319790
:10515000F1F700C00000D8CF8F929F92AF92BF921C
:10516000DF92EF92FF920F931F93CF93DF937C0117
:10517000CB01D22EDB01ED91FC910084F185E02D75
:1051800009951F928F9386EE91E09F938F930E94D3
:105190001403E80148018D0C911C0F900F900F90A3
:1051A0000F9080EEA82E81E0B82EC815D90561F0C9
:1051B00089911F928F93BF92AF920E9414030F9018
:1051C0000F900F900F90F1CF8DED91E09F938F9303
:1051D0000E9414030F900F90B8E082ED91E0DB1273
:1051E00006C0F80182818130A1F488EB91E09F93A1
:1051F0008F930E9414030F900F90DF91CF911F9116
:105200000F91FF90EF90DF90BF90AF909F908F90A5
:105210000895D701129688E001900D928A95E1F7E2
:105220000E94970CD7011B967C936E931A97E5CF3B
:105230003F924F925F926F927F928F929F92AF9226
:10524000BF92CF92DF92EF92FF920F931F93CF9373
:10525000DF9300D0CDB7DEB77C014DB65EB6DC0182
:105260005C968C9181111BC0312C832D0FB6F89464
:105270005EBE0FBE4DBE0F900F90DF91CF911F917C
:105280000F91FF90EF90DF90CF90BF90AF909F90E5
:105290008F907F906F905F904F903F9008950E9405
:1052A000970CF701808C918CA28CB38C68197909CA
:1052B0008A099B0997FDD8CF6701B12CA12C312C0D
:1052C000D70157968C918150990BA816B9060CF00E
:1052D0004DC06DB67EB6BFEFAB1ABB0AF601428574
:1052E000838590E081349105E0F59A8389838981F3
:1052F0009A81ADB7BEB7A81BB90B0FB6F894BEBF65
:105300000FBEADBFEDB7FEB731968F019E012F5F87
:105310003F4FD70116966C91169714968D919C91DC
:105320000E945E14382E811113C029813A812330E6
:10533000310570F0F70180899189009749F0DC010F
:10534000ED91FC910190F081E02D40E0B7010995CD
:105350000FB6F8947EBE0FBE6DBEB3E0CB0ED11C6F
:10536000AFCF20E430E03A832983C1CF0E94970C6D
:10537000F701258D620F711D811D911D608F718F49
:10538000828F938F72CFCF93109252041092510458
:1053900088EE93E0A0E0B0E080935304909354042F
:1053A000A0935504B093560485E691E09093500481
:1053B00080934F048FEF9FEF90935C0480935B0486
:1053C0008DE891E090936F0580936E0510927605BD
:1053D00081E0809377051092780580E795E09093BF
:1053E0007505809374051092700588E080937105AF
:1053F0008CE38093720510927305EEE6F5E0C1E050
:1054000080E795E01586C68717869487838735964B
:1054100025E0E93BF207B1F71092E40581E18093C2
:105420009F048FE495E00E941D0380E395E00E94B5
:105430001D0381E195E00E941D0382EF94E00E942C
:105440001D0387E991E09093E7048093E60490932D
:10545000DB048093DA049093CF048093CE0490937E
:10546000C3048093C20487E791E09093B2048093D1
:10547000B1048EE695E09093B4048093B304109247
:10548000C1041092B50488E08093B6049CE3909325
:10549000B704C093B8048093B90484E08093BA043D
:1054A0001092BB041092BC041092BD041092BE0472
:1054B0001092BF041092C004A4ECB5E0FD0190E08E
:1054C00080E021913191232B09F044C0880F991F6E
:1054D000FC01EC53FA4F81EB94E09183808387E7E2
:1054E00091E09093A1048093A0048EE695E09093C0
:1054F000A3048093A2041092B0041092A40488E044
:105500008093A5049CE39093A60491E09093A70454
:105510008093A80484E08093A9041092AA041092B6
:10552000AB041092AC041092AD041092AE04109231
:10553000AF0490E080E02D913D91232B89F4880FFA
:10554000991FFC01EC53FA4F80EA94E09183808329
:10555000CF91089501968031910509F0B2CFBFCF68
:1055600001968031910539F7F3CF1F920F920FB654
:105570000F9211248F939F93AF93BF938091410417
:10558000811113C080913D0490913E04A0913F048D
:10559000B09140044196A11DB11D80933D049093AC
:1055A0003E04A0933F04B0934004BF91AF919F91FC
:1055B0008F910F900FBE0F901F9018951F920F9212
:1055C0000FB60F9211242F933F934F935F936F93D6
:1055D0007F938F939F93AF93BF93EF93FF938091AC
:1055E000E10082FF09C08091E20082FF05C0809146
:1055F000E1008B7F8093E1008091DA0080FF1FC083
:105600008091D80080FF1BC08091DA008E7F80934C
:10561000DA008091D90080FFBFC080E189BD82E1BE
:1056200089BD09B400FEFDCF81E08093F502809131
:10563000DE02811104C00E9485060E94D00A80917A
:10564000E10080FF21C08091E20080FF1DC08091B9
:10565000E2008E7F8093E2008091E200806180937F
:10566000E2008091D80080628093D80019BC85E068
:105670008093F5028091E1028093DF021092E102B3
:1056800010923C040E94E01E8091E10084FF2FC034
:105690008091E20084FF2BC080E189BD82E189BD59
:1056A00009B400FEFDCF8091D8008F7D8093D80093
:1056B0008091E1008F7E8093E1008091E2008F7EF7
:1056C0008093E2008091E20081608093E20080910B
:1056D000EC02882309F466C084E08093F5021092FE
:1056E0003C040E94E01E8091DF028093E1028091E1
:1056F000E10083FF40C08091E20083FF3CC08091C5
:10570000E100877F8093E10082E08093F5021092B0
:10571000EC028091E1008E7F8093E1008091E200B5
:105720008E7F8093E2008091E20080618093E200AE
:1057300042E060E080E00E94700781E08093110108
:105740001092E0021092E10298E0E2EEF2E0DF0156
:105750001D929A95E9F710929D0210929E02109266
:105760009F021092A0021092A1021092A202109227
:10577000A30280931001FF91EF91BF91AF919F9190
:105780008F917F916F915F914F913F912F910F90EA
:105790000FBE0F901F90189519BC1092F502109231
:1057A000DE024DCF8091E30087FD02C081E095CFFE
:1057B00083E093CFCF93DF93CDB7DEB72A970FB6B1
:1057C000F894DEBF0FBECDBF84B7877F84BF0FB60E
:1057D000F894A89580916000886180936000109291
:1057E00060000FBE80E890E00FB6F89480936100EF
:1057F000909361000FBE82EB9DE090939B0180939C
:105800009A0186E091E0909346048093450480E1FC
:1058100092E00E947B020E9485060E94D00A789442
:1058200082E084BD93E095BD9AEF97BD80936E00B2
:1058300080914404816080934404269A0E94AC0EB7
:10584000219A229A2398209A80E58CBD81E08DBD13
:10585000259868E188E80E94D20E60E288E70E94FD
:10586000D20E60E088E70E94D20E10E000E088E6E9
:105870000E94E50E0F5F1F4F80FF1CC061EC88ED9A
:105880000E94D20E60E280ED0E94D20E64E088EEAB
:105890000E94D20E88EE0E94E50E82FFFBCF0E948E
:1058A0008B1060E288EC0E94D20E61E080E80E94DA
:1058B000D20E03C00F3F1007D1F686EE94E090930E
:1058C000600580935F058AED94E090934105809395
:1058D00040058EEC94E0909322058093210582ECA4
:1058E00094E090930305809302058091F502843043
:1058F00009F0DBC00E94A30C882309F4D6C08EEF08
:1059000091E00E947B0280EF91E00E947B0277246D
:105910007A9423E0622E30E1532E48E1C42ED12C3C
:105920008091F502853009F4C3C00E94021F0CEB80
:1059300012E0412C842D0E94E8104C01F801A08057
:10594000B1808A159B0571F1312CEE24E394F12C82
:10595000A824B924C5018E219F21892BE9F03E821C
:105960004F8221E0C70188219921892B09F420E089
:1059700028870E94B60C8160782F9A8789874E818C
:105980005F8168858A850E944127F8018081918125
:105990008E259F25918380833394EE0CFF1CF0E1CC
:1059A0003F12D8CF43940E5F1F4F40E14412C2CF45
:1059B00079827A821B820E94B60C8160782F9D8347
:1059C0008C8349815A816B818D810E94412720916E
:1059D0004704309148044FB7F89480913D0490916A
:1059E0003E04A0913F04B09140044FBFFC01E21B74
:1059F000F30B9F018091430442E350E0811102C008
:105A00004CE251E02417350780F090914A04109140
:105A10004B04F0904C0400914D04911183C011117E
:105A200046C1F11044C1011142C10E947906909112
:105A3000BB02891731F00E9479068093BB020E9455
:105A40008E1B2091E4003091E5008091DC02909162
:105A5000DD022817390731F18091E4009091E500CB
:105A60009093DD028093DC020E94A30C8823D1F086
:105A70008091F5028430B1F48091E9008F709091AB
:105A8000EC0090FFBDC090E8892B6092E9009091F6
:105A9000EB0090FF04C09091EE0097FDCFC08F7097
:105AA0008093E9000E94A2073BCF0E94A2071DCF6E
:105AB0008091F502843011F11092410480E40FB618
:105AC000F894A895C09260000FBE8093600083B7E1
:105AD000817F846083BF83B7816083BF789488951A
:105AE00083B78E7F83BF0FB6F894A895809160002E
:105AF000886180936000109260000FBE8091EB027D
:105B0000882369F00E94021F10E0812F0E94E81094
:105B1000892B09F0B7C01F5F1031B9F701CF0E9480
:105B2000021FFECE8F3F19F08F5F8093430419163A
:105B300024F40E94FD0380934A0480914A0487FF65
:105B400005C00E94FD03819580934A04111624F438
:105B50000E94FD0380934B0480914B0487FF05C096
:105B60000E94FD03819580934B0460914A04662353
:105B700031F110914B04112311F1062E000C770B1B
:105B8000880B990B0E94BE2E23E333E343E35FE3CC
:105B90000E944B2F0E94862E60934A04612F110FA2
:105BA000770B880B990B0E94BE2E23E333E343E36C
:105BB0005FE30E944B2F0E94862E60934B041F14BC
:105BC00024F40E94DB0380934C0480914C0487FFF3
:105BD00005C00E94DB03819580934C04101624F4C9
:105BE0000E94DB0380934D0480914D0487FF05C024
:105BF0000E94DB03819580934D040E94451E15CFC2
:105C000090E042CFE0910101F0910201E90FF11D16
:105C100020819F5F3091050193239093040120938D
:105C2000F1009091E80095FD09C09091E80090FF87
:105C300005C09091E8009E779093E8009091040150
:105C400020910301291721F02091E80025FDDACFEA
:105C50002091F3009091F200322F292F232B09F489
:105C60001ECF9091E80090FF1ACF9091E80095FD2B
:105C700006C09091E8009E779093E80010CF1092B4
:105C8000F100F3CF59BC82E189BD09B400FEFDCF1C
:105C90008091D8008F7D8093D8008091E000826051
:105CA0008093E0008091E00081FDFCCF39CE8F3FF2
:105CB00009F03ACF4BCF78941F920F920FB60F9204
:105CC00011248F939F93AF93BF9380913D04909144
:105CD0003E04A0913F04B09140040196A11DB11D66
:105CE00080933D0490933E04A0933F04B0934004FE
:105CF000BF91AF919F918F910F900FBE0F901F900A
:105D000018950E94F92E08F481E008950E948D2EC6
:105D10006894B1110C94402F08950E94252F88F0AB
:105D20009F5798F0B92F9927B751B0F0E1F0660F5F
:105D3000771F881F991F1AF0BA95C9F714C0B130A0
:105D400091F00E943F2FB1E008950C943F2F672FF0
:105D5000782F8827B85F39F0B93FCCF386957795CF
:105D60006795B395D9F73EF49095809570956195B8
:105D70007F4F8F4F9F4F0895E89409C097FB3EF4E3
:105D800090958095709561957F4F8F4F9F4F992388
:105D9000A9F0F92F96E9BB279395F6958795779506
:105DA0006795B795F111F8CFFAF4BB0F11F460FFC6
:105DB0001BC06F5F7F4F8F4F9F4F16C0882311F01E
:105DC00096E911C0772321F09EE8872F762F05C032
:105DD000662371F096E8862F70E060E02AF09A95CD
:105DE000660F771F881FDAF7880F9695879597F9C2
:105DF0000895990F0008550FAA0BE0E8FEEF16165C
:105E00001706E807F907C0F012161306E407F507AE
:105E100098F0621B730B840B950B39F40A2661F022
:105E2000232B242B252B21F408950A2609F4A140C5
:105E3000A6958FEF811D811D089557FD9058440F41
:105E4000551F59F05F3F71F04795880F97FB991FD9
:105E500061F09F3F79F08795089512161306140696
:105E6000551FF2CF4695F1DF08C016161706180623
:105E7000991FF1CF86957105610508940895E894FE
:105E8000BB2766277727CB0197F908950E94F92E43
:105E900008F48FEF08950E945E2F0C94CF2F0E947C
:105EA000C12F38F00E94C82F20F0952311F00C94D8
:105EB000B82F0C94BE2F11240C94402F0E941D2F3C
:105EC00070F3959FC1F3950F50E0551F629FF0014D
:105ED000729FBB27F00DB11D639FAA27F00DB11D66
:105EE000AA1F649F6627B00DA11D661F829F2227EF
:105EF000B00DA11D621F739FB00DA11D621F839F76
:105F0000A00D611D221F749F3327A00D611D231F4B
:105F1000849F600D211D822F762F6A2F11249F5799
:105F200050409AF0F1F088234AF0EE0FFF1FBB1F9C
:105F3000661F771F881F91505040A9F79E3F51055B
:105F400080F00C94B82F0C94402F5F3FE4F3983E00
:105F5000D4F3869577956795B795F795E7959F5F05
:105F6000C1F7FE2B880F911D9695879597F9089597
:105F700097F99F6780E870E060E008959FEF80ECFC
:105F8000089500240A94161617061806090608959F
:105F900000240A9412161306140605060895092E05
:105FA0000394000C11F4882352F0BB0F40F4BF2B74
:105FB00011F460FF04C06F5F7F4F8F4F9F4F0895B4
:105FC00097FB072E16F4009407D077FD09D00E94A6
:105FD000FA2F07FC05D03EF4909581959F4F0895C8
:105FE000709561957F4F0895EE0FFF1F0590F49116
:105FF000E02D0994AA1BBB1B51E107C0AA1FBB1FC0
:10600000A617B70710F0A61BB70B881F991F5A9544
:10601000A9F780959095BC01CD010895F894FFCF24
:10602000059C010000FF310B7A284C280C28D4274E
:106030000101FF66756C6C006C6F7700000000005A
:10604000851100000000A612000000002F0E407F06
:10605000224D01CE00AC0047026002790200000030
:10606000000619C5138F0E18298C0EC413C213878E
:106070000E820E770EDC10D910300EFEFF00006D80
:106080000E000000001F0E050E260E250E2C0E29F8
:106090000E290E00000000B317C5136F0B9F1D964D
:1060A0000B5817C213910B950C00000000620C0DE9
:0A60B0000CEB0B00000000AC280010
:106800008800EA44E944E244040005000600070069
:10681000080009000A000B000C000D000E000F001C
:1068200010001100120013001400150016001700CC
:10683000180019001A001B001C001D001E001F007C
:10684000200021002200230024002500260027002C
:10685000280029002A002B002C002D002E002F00DC
:10686000300031003200330034003500360037008C
:10687000380039003A003B003C003D003E003F003C
:1068800040004100420043004400450046004700EC
:10689000480049004A004B004C004D004E004F009C
:1068A000500051005200530054005500560057004C
:1068B000580059005A005B005C005D005E005F00FC
:1068C00060006100620063006400F1A18500670060
:1068D000680069006A006B006C006D006E006F005C
:1068E0007000710072007300890087008A008B00BD
:1068F000E000E100E200E300E400E500E600E7007C
:106900000100010001000100EA4401000100E2442D
:106910000100010001000100460001004A004B0097
:10692000010001004700480001000100E9440100A6
:106930000100010001000100010001003A003B00DC
:106940003C003D003E003F0040004100420043004B
:10695000010035004C0001000100440045005200D8
:1069600049000100010050004F0029004D004E0079
:1069700051000100010001000100010001000100BF
:1069800001000100010001000100010001000100FF
:1069900000E00100010001000100010001004D00C4
:1069A0004A004E004B0001000100010001000100FF
:1069B00001000100010001000100010001000100CF
:1069C00001000100010001000100010001000100BF
:1069D00001000100010001000100010001000100AF
:1069E0000100010001000100490001000100010057
:1069F000010001000100010001000100010001008F
:00000001FF
